:10000000020A458CC3AF058FC4A2AF92D5C2AF75AB
:0C001000C65A75C6A50000A2D592AF220A
:100023000208A4EFD394077480948040037FFF22D7
:100033001204D1FED394037480948040037FFF2283
:10004300EF7044EE700B9000011204EAF4529352E5
:10005300941204D16401700B9000011204EA4293DC
:10006300F452941204D1FE6402700A900001120447
:10007300EA42934294EE6403700D9000011204EA85
:10008300FEF45293EE4294EF640170461204D1FEE3
:10009300700B9000011204EAF452915292EE640143
:1000A300700B9000011204EA4291F452921204D1AF
:1000B3006402700A9000011204EA4291429212040F
:1000C300D16403700D9000011204EAFEF45291EE24
:1000D3004292EF640270461204D1FE700B9000014D
:1000E3001204EAF452955296EE6401700B900001EB
:1000F3001204EA4295F452961204D16402700A90F3
:1001030000011204EA429542961204D16403700D71
:100113009000011204EAFEF45295EE4296EF640356
:1001230070461204D1FE700B9000011204EAF452DF
:10013300B152B2EE6401700B9000011204EA42B1B5
:10014300F452B21204D16402700A9000011204EA5C
:1001530042B142B21204D16403700D900001120443
:10016300EAFEF452B1EE42B2EF640470461204D1D7
:10017300FE700B9000011204EAF452B352B4EE6421
:1001830001700B9000011204EA42B3F452B412045A
:10019300D16402700A9000011204EA42B342B4121D
:1001A30004D16403700D9000011204EAFEF452B30B
:1001B300EE42B4EF640570461204D1FE700B90005A
:1001C300011204EAF452C952CAEE6401700B9000A2
:1001D300011204EA42C9F452CA1204D16402700A39
:1001E3009000011204EA42C942CA1204D1640370A6
:1001F3000D9000011204EAFEF452C9EE42CAEF6404
:100203000670461204D1FE700B9000011204EAF44A
:1002130052CB52CCEE6401700B9000011204EA42FF
:10022300CBF452CC1204D16402700A900001120480
:10023300EA42CB42CC1204D16403700D9000011248
:1002430004EAFEF452CBEE42CCEF64077049120489
:10025300D1FF7E00700B9000011204EAF452E152C8
:10026300E2EF64014E700B9000011204EA42E1F4E4
:1002730052E21204D16402700A9000011204EA42AD
:10028300E142E21204D16403700D9000011204EA0A
:10029300FFF452E1EF42E27F0022120A2712099A89
:1002A300D2AF7BFF7A0A795B120A147BFF7A0A7951
:1002B3008D120A147BFF7A0A79C6120A147BFF7A1D
:1002C3000B7901120A147F017E001209EAD3E52299
:1002D30094007480948040EE1522E52270E8F508BE
:1002E300E508C39521501474002508F582E4340011
:1002F300F583E0FF120A51050880E5750CFFC3E59D
:100303002194087480948050030204BE900001E09D
:10031300642060030204BEF508C3E50894087480F2
:100323009480502D74002508F582E43400F583E0B1
:10033300FFC394614017EFD3947A5011EF24E0FF89
:1003430074002508F582E43400F583EFF005088096
:10035300C81208038E0A8F0BE4FCFDFB7AF8F9F848
:10036300D31205F750030204BE900000E0B4451019
:10037300AF0BAE0A120A017BFF7A0B793A02041B18
:10038300900000E064576003020421900008E064D9
:10039300206003020421E52124F7F509D394647452
:1003A30080948040037509647B017A007909751292
:1003B30000850913AF0BAE0A1209327BFF7A0B7962
:1003C30047120A14C3E5099464748094804015E5C8
:1003D3000975F064842430FF120A51E50975F0644D
:1003E3008485F009C3E509940A748094804015E577
:1003F3000975F00A842430FF120A51E50975F00AE1
:100403008485F009E50975F00A84E5F02430FF12CC
:100413000A517BFF7A0B794E120A140204BB900037
:1004230000E0645260030204BE900008E0642060B0
:10043300030204BE1209C38F09D3EF94647480943A
:10044300804003750964D3E5099400748094804067
:100453006A7BFF7A0B7957120A14E50975F00A844F
:100463002430FF120A51E50975F00A84E5F02430BF
:10047300FF120A517BFF7A0B795C120A147B017A13
:10048300017900751200850913AF0BAE0A120969D1
:10049300E4F508E508C39509501474002508F582AE
:1004A300E43401F583E0FF120A51050880E57F0D6E
:1004B300120A517F0A120A51E4F50CE50C60097B1C
:1004C300FF7A0B796F120A14E4F5210202C9BB010A
:1004D3000689828A83E0225002E722BBFE02E322DE
:1004E30089828A83E49322BB010CE58229F582E5A4
:1004F300833AF583E0225006E92582F8E622BBFE23
:1005030006E92582F8E222E58229F582E5833AF5B8
:1005130083E49322BB010689828A83F0225002F787
:1005230022BBFE01F32275F008758200EF2FFFEE68
:1005330033FECD33CDCC33CCC58233C5829BED9A0C
:10054300EC99E58298400CF582EE9BFEED9AFDEC6A
:1005530099FC0FD5F0D6E4CEFBE4CDFAE4CCF9A8B0
:100563008222B800C1B90059BA002DEC8BF084CFB8
:10057300CECDFCE5F0CBF97818EF2FFFEE33FEED8F
:1005830033FDEC33FCEB33FB10D703994004EB99B9
:10059300FB0FD8E5E4F9FA227818EF2FFFEE33FECC
:1005A300ED33FDEC33FCC933C910D7059BE99A4001
:1005B30007EC9BFCE99AF90FD8E0E4C9FAE4CCFB19
:1005C3002275F010EF2FFFEE33FEED33FDCC33CC6D
:1005D300C833C810D7079BEC9AE899400AED9BFDF6
:1005E300EC9AFCE899F80FD5F0DAE4CDFBE4CCFA09
:1005F300E4C8F922EB9FF5F0EA9E42F0E99D42F050
:10060300EC6480C864809845F022EB9FF5F0EA9E85
:1006130042F0E99D42F0E89C45F022E8600FECC30C
:1006230013FCED13FDEE13FEEF13FFD8F122BB0114
:100633000DE58229F582E5833AF58302066E5007BC
:10064300E92582F8020661BBFE07E92582F8020666
:100653007AE58229F582E5833AF583020687E6FB8C
:1006630008E6F908E6FA08E6CBF822E0F8A3E0F991
:10067300A3E0FAA3E0FB22E2FB08E2F908E2FA08AE
:10068300E2CBF822E493F8740193F9740293FA74B9
:100693000393FB228B168A178918EF640160030208
:1006A3000800751D01F51EF51FF520F521F522F54E
:1006B30023FFEFC3948074809480500F74802FF5D0
:1006C30082E43400F583E4F00F80E7E4FFEFC394A2
:1006D3008074809480500F74002FF582E43400F509
:1006E30083E4F00F80E7AB16AA17A9181204D1FF11
:1006F300E598543F4FF598EF64C06008EF6440609D
:10070300030207AF9000021206317F007E607D5422
:100713007C001205658F1C8E1B8D1A8C19E4FFFE5D
:100723007D01FCAB1CAA1BA91AA819C312060D4014
:10073300037FFF22C3E4951CF51CE4951BF51B7492
:1007430001951AF51AE49519F519AB16AA17A91804
:100753009000011204EA64027026538EEF438E0167
:10076300538EF7438E04AF1CAE1BAD1AAC19780839
:1007730012061E8FD6851CD753AFFB438E1080669F
:10078300C28E538EFE5389BF5389CF438E40AF1C15
:10079300AE1BAD1AAC19780812061E8F8D851C8B03
:1007A300C2AB5389BF538FFDD28E803AAB16AA17C3
:1007B300A9181204D1FF7E0070149000081204EAF5
:1007C30064017005438E20801D538EDF8018EF6413
:1007D300804E70129000081204EA6401700543878A
:1007E30080800353877FAB16AA17A91890000712BE
:1007F30004EA7004C29C8002D29C7F00227FFF2205
:10080300E4FBFA900002E064307044A3E0645870A3
:100813003E7C04ECC3940874809480502D74002CA7
:100823001208F2AD07EDC3941074809480400280E7
:100833001EEBC4F8540FC868FFEAC454F048FEED39
:100843007A002FFBEA3EFA0C80C9AE02AF03227E88
:10085300FF7FFF22EFFBD39401748094805009EB58
:100863007004C2AC8002D2ACEDFF7E00D39403745B
:100873008094805029EF700553B7EFC2BCEF640139
:100883004E700553B7EFD2BCEF64024E700543B709
:1008930010C2BCEF64034E700543B710D2BC7F0097
:1008A30022C0E0C083C082C0D075D000C00730989A
:1008B30028C298E5237022C3E52194807480948034
:1008C3004003752100AF21052174002FF582E43424
:1008D30000F583E599F0752205309905C2997520D5
:1008E30000D007D0D0D082D083D0E03274002DF571
:1008F30082E43400F583E0FFEFC39430400CEFD380
:1009030094395006C3EF9430FF22EFC39441400B58
:10091300EFD394465005EF24C9FF22EFC3946140FF
:100923000BEFD394665005EF24A9FF227FFF22AD7E
:1009330007AC0675C78075F51675C5028CC3AF0580
:100943008FC41204D1F5C21200090DBD00010C744D
:100953000129F9E43AFAE513151370021512144547
:100963001270D9020A37AD07AC0675C78075F51644
:1009730075C501120003E5C21205170DBD00010C78
:10098300740129F9E43AFAE51315137002151214E8
:10099300451270DF020A37750D40750E017512009E
:1009A3007511C2751001750F00751401E4F515FB7F
:1009B3007A00790D7F011206977D017F01020857A6
:1009C300E4FE7D09EDC39521501A1208EFEFC3949D
:1009D3000A74809480500D1208EFEE75F00AA42F6C
:1009E300FE0D80E0AF06227DA37C08ED1D70011C87
:1009F300144C70F7EF1F70011E144E70EA22AD07FE
:100A0300AC0675C78075F51675C503120003020A97
:100A1300371204D1FF600C120A51740129F9E43A28
:100A2300FA80EE22750E03E4F50DFB7A00790D7F53
:100A330003020026E4F5C7F5C5F5C675C3FF75C403
:100A4300FF22787FE4F6D8FD75812302029D8F99FA
:100A5300752001E52070FC2253544338CFB5C1D033
:100A6300B5A5C6ACBBFA454550524F4DB2E2CAD408
:100A7300B3CCD0F2A3ACB4AEBFDAC3FCC1EEC9E8C9
:100A8300D6C3C8E7CFC23A0D0A00452030783030CC
:100A93003430202020202020202020202020202D22
:100AA3002D3E20B6D4307830303430B5D8D6B7C9DF
:100AB300C8C7F8C4DAC8DDBDF8D0D0B2C1B3FD2EC3
:100AC3000D0A00572030783030343020313233343F
:100AD30035363738393020202D2D3E20B6D43078A6
:100AE30030303430B5D8D6B7D0B4C8EBD7D6B7FB8F
:100AF300313233343536373839302E0D0A0052202F
:100B03003078303034302031302020202020202015
:100B13002020202D2D3E20B6D4307830303430B50F
:100B2300D8D6B7B6C1B3F63130B8F6D7D6BDDAC426
:100B3300DAC8DD2E0D0A00B2C1B3FDB3C9B9A6A34D
:100B4300A10D0A00D2D1D0B4C8EB00D7D6BDDAA329
:100B5300A10D0A00B6C1B3F600B8F6D7D6BDDAC404
:100B6300DAC8DDC8E7CFC2A3BA0D0A00C3FCC1EEE1
:090B7300B4EDCEF3A3A10D0A00BC
:00000001FF
